:100000002CC1000045C1000043C1000041C10000F7
:100010003FC100003DC100003BC1000039C10000EC
:1000200037C1000035C1000033C10000D0C200005C
:100030003AC300002DC100002BC1000029C10000FF
:1000400027C1000025C1000023C1000021C100001C
:100050001FC100001DC100001BC1000019C100002C
:1000600017C1000015C1000013C1000011C100003C
:100070000FC1000000888A41828463428900000029
:100080003A6040802C8657590000001D0605103745
:1000900085543F000000811B191136385D45000072
:1000A000004C16090B0E3328440000003B04070ADD
:1000B0000D0F345F0000003C1A151C0C13305E005D
:1000C00000002B14081718122F2A000000551F21BA
:1000D0002325272E310000001E202224262D3556F0
:1000E00000000029625C5B5A433D3E0000000000B6
:1000F0000000000000888A418284514E890000007F
:100100003A6040802C504F4D0000001D060510370E
:10011000854B3F000000811B191136385245000005
:10012000004C16090B0E33284A0000003B04070A56
:100130000D0F345F0000003C1A151C0C13305E00DC
:1001400000002B14081718122F2A000000551F2139
:100150002325272E310000001E202224262D35566F
:1001600000000029625C5B5A433D3E000000000035
:1001700000000000245265766973696F6E3A20347E
:1001800034323520240000010000BD0112000200BD
:1001900000CF012200220000F1013F00210000E118
:1001A00001090003000030020401030904340210B5
:1001B00002030904460212000001C10600120100F8
:1001C0000200000020C0167C0400010102000109A9
:1001D000022200010100C0320904000001030101F4
:1001E00000092111010001223F00070583030800D7
:1001F0000105010906A10175019508050719E02906
:10020000E7150025018102950175088103950575A3
:1002100001050819012905910295017503910395BE
:10022000067508150025680507190029688100C0B2
:100230000403090410034D00660067004E006100CE
:100240006D006500000012034B006500790062003C
:100250006F00610072006400000011241FBECFEF28
:10026000D2E0DEBFCDBF11E0A0E0B1E0EEEBF9E0FF
:1002700002C005900D92A230B107D9F711E0A2E0BB
:10028000B1E001C01D92AD32B107E1F7F7D095C3DF
:10029000B7CEFB01DC0104C08D910190801921F4DF
:1002A00041505040C8F7881B990B08955E9825E38C
:1002B0002A95F1F75E9AE0E9F1E03197F1F760E015
:1002C00070E0BAE2A5ED19C056955D984B2F4A959E
:1002D000F1F75D9A4A2F4A95F1F74C9B50682F5FD2
:1002E0003F4F2830310581F7FC01E60FF71F50839F
:1002F0006F5F7F4F6031710521F050E020E030E00A
:10030000E3CF0895CF93DF93C4E7D1E001C02196F6
:10031000FE019491992369F0892F80538A30B8F7B0
:10032000903311F487E202C0892F835160E042D1FB
:10033000EECFDF91CF910895E4E2F1E003C0819127
:10034000882389F481E0E932F807C9F78091230115
:10035000853019F0893139F405C01092D8000C9419
:1003600000180895CFCF0895AF92BF92CF92DF9239
:10037000EF92FF920F931F93CF93DF93EC0100E076
:10038000FF2464E770E053E2A52E51E0B52E46E06D
:10039000E42E31E0C32ED12C10922201F5018E2DD6
:1003A00011928A95E9F750E080E020E030E0FE010C
:1003B000E20FF31FB081A0912201482F182F185F80
:1003C000FB01E40FF11D4F5F8491B0FF2FC0882324
:1003D00069F187FF23C090E08F7790708830910596
:1003E00049F08930910544F08930910569F00A9708
:1003F000E9F411C001E01AC0F60102C0EE0FFF1FC0
:100400008A95E2F7AE2B12C0F0E064377F0771F4F3
:1004100064EF70E0C1CFFF24F39408C0563030F48D
:10042000E52FF0E0ED5DFE4F80835F5F411711F037
:10043000B695C6CFA09322012F5F3F4F20313105E3
:1004400011F0842FB4CF002311F076DF01C06AD001
:100450008091290190E0969587958170F81619F0A2
:1004600089E360E0A7D0DF91CF911F910F91FF90BA
:10047000EF90DF90CF90BF90AF900895CF93DF9330
:1004800080E8809361001092610080E68AB980E77D
:100490008BB931D044D08823E9F380E395E720E994
:1004A00031E0F9013197F1F70197D9F780E1E2E006
:1004B000F1E0DF011D928A95E9F7C0E4DCE982E111
:1004C00091E0F4DE82E191E062E071E040E150E031
:1004D000E0DE009761F082E191E046DFA2E0B1E06A
:1004E000E2E1F1E080E101900D928150E1F7CE016F
:1004F0000197F1F7E4CF80EA8093D80086E089BDC8
:1005000009B400FEFDCF80E88093D8001092E0008F
:1005100010922A018CE08093E200789408958091F3
:100520002A01089580912A01882309F441C02FB738
:10053000F89483E08093E9009091E4009E5C33E0BE
:100540008091E80085FD0EC02FBF80912A0188238D
:1005500079F18091E400891759F12FB7F89430931D
:10056000E900EECF809122018093F1001092F1001A
:10057000809123018093F100809124018093F10008
:10058000809125018093F100809126018093F100F4
:10059000809127018093F100809128018093F100E0
:1005A0008AE38093E80010922B012FBF80E008952A
:1005B0008FEF08956093220180932301B3DF882396
:1005C00029F41092220110922301ACCF08951F92BA
:1005D0000F920FB60F9211242F938F939F938091B8
:1005E000E1001092E100982F83FF0FC01092E90004
:1005F00081E08093EB001092EC0082E28093ED00AA
:1006000088E08093F00010922A0192FF44C080910C
:100610002A01882309F43FC0209100012223D9F147
:1006200080912C018F5F80932C0190E083709070FB
:10063000892B89F583E08093E9008091E80085FFAC
:100640002AC080912B018F5F80932B01821719F5AF
:1006500010922B01809122018093F1001092F10001
:10066000809123018093F100809124018093F10017
:10067000809125018093F100809126018093F10003
:10068000809127018093F100809128018093F100EF
:100690008AE38093E8009F918F912F910F900FBE76
:1006A0000F901F9018951F920F920FB60F92112462
:1006B0000F931F932F933F934F935F936F937F936A
:1006C0008F939F93AF93BF93EF93FF931092E900A3
:1006D0008091E80083FF5BC14091F1003091F1000F
:1006E0008091F100682F70E02091F100922F80E05E
:1006F000682B792B8091F100A82FB0E02091F100B8
:10070000922F80E0A82BB92B1091F1000091F100FD
:1007100082EF8093E800363009F05AC02DE831E0CE
:10072000A90145505040F90137978591949186175A
:10073000970701F5FA01859194918A179B07D1F4E7
:100740009A012E5F3F4FF901659174912E5F3F4FE3
:10075000F9014491212F30E0902F80E0282B392B94
:100760002F3F310519F010F02FEF30E0241758F427
:10077000422F09C0295F3F4F495F5F4FF1E02E3B99
:100780003F0789F604C15EEF8091E800282F30E032
:10079000C90185709070892BB9F322FDFBC0342FFD
:1007A000413208F030E2232FCB0106C0FC01019654
:1007B000E491E093F10021502223C1F7630F711DF2
:1007C000431B5093E8004423F9F63032E9F2E2C0CB
:1007D000353061F48EEF8093E8008091E80080FF6F
:1007E000FCCF862F80688093E300D4C0393031F588
:1007F000442309F071C060932A018EEF8093E800D2
:1008000087EB91E021E02093E900FC010196E4915F
:10081000E093EB00EE2369F0AC014F5F5F4FFC010A
:1008200084918093EC00CA010196FA0134913093CF
:10083000ED002F5F253039F78EE149C0383051F493
:10084000403809F049C08091E80080FFFCCF8091DA
:100850002A017BC03323D1F48091E80080FFFCCFD4
:10086000423811F080E00DC0A093E9008091EB00C8
:1008700090E025E0969587952A95E1F78170109292
:10088000E9008093F1001092F1007DC0313011F049
:10089000333011F5423001F561157105E9F42A2F65
:1008A0002F77822F81508430B8F48EEF8093E80048
:1008B0002093E900333009F46AC089E18093EB00AA
:1008C00081E090E002C0880F991F2A95E2F780939B
:1008D000EA001092EA005EC0AB2B09F058C0413A22
:1008E000B9F5313009F58091E80080FFFCCF8091A7
:1008F00022018093F1001092F100809123018093F6
:10090000F100809124018093F10080912501809372
:10091000F100809126018093F1008091270180935E
:10092000F1008091280111C0323039F48091E80043
:1009300080FFFCCF8091000108C0333041F58091E9
:10094000E80080FFFCCF809101018093F1001BC083
:100950004132E9F4393061F48091E80082FFFCCF44
:100960008091F100809329018BEF8093E8000BC008
:100970003A3029F47093000110922B0104C03B30EF
:1009800031F4609301018EEF8093E80003C081E2AF
:100990008093EB00FF91EF91BF91AF919F918F9169
:1009A0007F916F915F914F913F912F911F910F9187
:0E09B0000F900FBE0F901F901895F894FFCF78
:0209BE007D01B9
:00000001FF
